:020000040000FA
:10000000000080310000C4288031D92823009100ED
:10001000230015141308910A0319920A20000800FE
:10002000230093000430950055309600AA309600C6
:1000300095149518FE331511910A0319920A2000A0
:10004000080008308501AB002418AB20210884008B
:1000500022082419BA20241DBC202008840023096A
:100060008417800520088400A60CA50C0008230432
:10007000031C230680003F20AB0BF433080021084B
:100080008400220880060000003200320032800620
:100090000800A801A700FF30A707031CA807031C3E
:1000A00008000330A600E5305720F533A601FB3EDB
:1000B000A500A609FF30031C0332A5070318FD3372
:1000C000A5070000A60FF933000008000038031947
:1000D0001532AD002508840026188317A601A50156
:1000E000AD1B08320008A500AD1C0832840A0008C8
:1000F000A60004327F200005031DA50A0800013078
:100100002D180935AD180935AD1809352D19090E09
:100110000800013EAC000A30A700A8019320AC0BF8
:10012000FD3329080800AA01A9011030AB00260DF3
:10013000A90DAA0D2708A9022808AA3B0318053211
:100140002708A9072808AA3D0310A50DA60DAB0B8B
:10015000EE3325080800A701A8010432A60CA50C5F
:10016000A70DA80DFF3E0318F9332808A60027089D
:10017000A500080080040332FF3A80050132FF3AEF
:1001800084178005200008007A30210099002200A1
:1001900091019301073021009E0023008C018E0104
:1001A00021009517CE308C0047308E002000823120
:1001B000922A20000B1164309500B60A6430360292
:1001C0008031031DF728B601B20380318C18F42862
:1001D000B2088031031DF228B3033C30B20033086B
:1001E000B50034148031F7283208B5003414090002
:1001F00080310C1EFC280C120A30350281310318A4
:100200003C293508A700093C8131031C39292735D1
:10021000A70781311921A500A70A81311921A6005C
:10022000A70A81311921803166202508B10081316A
:10023000392927080B00EB3400340034283400340B
:100240000034B33400340034BA3400340034783429
:1002500000340034DA3400340034DB340034003449
:10026000E83400340034FB3400340034FA34003411
:100270000034B0018131CC290A30350281310318B4
:1002800043290301031D0130AE0064303502013003
:1002900003180030AE0581310319CC29A6013508B9
:1002A000A500003080318920B1003108A700093C49
:1002B0008131031C8D292735A70781316D21A500C8
:1002C000A70A81316D21A600A70A81316D218031F5
:1002D00066202508B10081318D2927080B00EB34F9
:1002E00000340034283400340034B3340034003493
:1002F000BA3400340034783400340034DA34003452
:100300000034DB3400340034E83400340034FB348F
:1003100000340034FA3400340034A6013508A50056
:10032000013080318920B0003008A700093C8131BC
:10033000031CCC292735A7078131AC21A500A70ACA
:100340008131AC21A600A70A8131AC218031662021
:100350002508B0008131CC2927080B00D7340034A0
:100360000034143400340034CD34003400345D34AF
:10037000003400341E34003400345B340034003464
:10038000DB3400340034173400340034DF340034FC
:1003900000345F34003400348E120A30803149203A
:1003A0000E30A0000830A3000E30A1001030A200D3
:1003B0000130A4003108A500803121203008A500BB
:1003C000803121200D30890BFE3300008E16341051
:1003D00008008131B418F729643095000B118B1691
:1003E0008B17B41421008C1220008C16341081312C
:1003F0000C19FE29643080314920F933080082311C
:10040000B41C0A2A0B118B128B13B41021008C120E
:1004100020008C128231B22A8231B418492A8231EA
:100420008C182E2A64303302823103181A2AB30A38
:100430008231212A643033028231031D212A633044
:10044000B3003C30B2003308B50002302300910005
:1004500020003308803110208231472A6430320274
:1004600082310318362AB20A82313D2A64303202C0
:100470008231031D3D2A6330B200B3013208B5005A
:10048000013023009100200032088031102080319B
:10049000F82082318E18502A643080314920F93397
:1004A00008008231B4188A2A82318C18712AB30864
:1004B000823103195E2AB3038231642AB308823180
:1004C000031D642A0130B3003C30B2003308B5008C
:1004D0000230230091002000330880311020823147
:1004E000882AB20882310319782AB20382317E2A1F
:1004F000B2088231031D7E2A0130B200B3013208F6
:10050000B500013023009100200032088031102016
:100510008031F82082310E18912A643080314920D0
:10052000F933080023308500DF308400800101307A
:1005300084020030853B1F300502031DF733210084
:100540008C1220008C12B001B10121000C1220008D
:100550000C16B501B201B30121001514951415153F
:1005600095119512200082318C18C22A02308031F8
:100570000620B3003C30B2003308B5008031F820CB
:100580008231CB2A013080310620B200B30132081B
:10059000B5008031F8200B118B128B13B41034107E
:1005A00082310C19D52A8131E92182318E18DA2A5B
:1005B00082310C2282310E18DF2A82315122003022
:1005C000B4180130AE00003034180130AE0582316D
:1005D0000319F12A8031F8203410B508813103194C
:0605E000FF29DE33FF33AA
:020000040001F9
:02000E0004F9F3
:02001000FFDE11
:06E0000000001400050001
:00000001FF
